:020000020000FC
:0400000009C05CC017
:020008008CC0AA
:10000C0076C081C08BC0B0C10FEF07BB0FEF08BB30
:10001C0008E304BB07E005BB0BEF01BB00E002BB30
:10002C000FE50DBF04E00EBF21E011243324662739
:10003C0077278827AA27BB27CC27DD2703E0202E8C
:10004C00442755270FEB802E902EA02EB02EC02EBD
:10005C00D02EE02EF02E002700936000009361005C
:10006C0000936400009365000FEF0093620000930F
:10007C006300009366000093670004E003BF00E098
:10008C000FBD03E00EBD00E00BBD00E10ABD00E0BA
:10009C0009BD00E408BD04E005BD0DE509BF01E89C
:1000AC0005BF00E40BBF00E808B978948895FECF33
:1000BC00000090B39470941509F41895492E92FF92
:1000CC0007C06CB57DB56031730580F034BC1895F4
:1000DC0064B5683058F03DBC3CBC603830F06624E8
:1000EC00772455241124882701C0862F1895883031
:1000FC0048F092FD07C0660C771C551C1394803297
:10010C0008F06394189592FD05C00CD066247724F2
:10011C0055241124189501E804BD18950FEF3DBC2A
:10012C000CBD189508E1101609F401D0089583014F
:10013C00102702951027012F169516950127102FC1
:10014C00169501270170172D12951170101709F0D3
:10015C000895172D109550945694179556941795FD
:10016C00569417955694179556941795072D077016
:10017C001615500609F0089573FC0BC0A3015770B7
:10018C0040936800509369000FD0AB9AA0E7B7E199
:10019C000AC0A301577040936A0050936B0074D04F
:1001AC00AC9AC0E7D7E1089510916300009162000A
:1001BC004017510720F45093630040936200109154
:1001CC006100009160000417150720F45093610042
:1001DC004093600020FC04C0509163004091620089
:1001EC0021FC04C05091610040916000413B04E04F
:1001FC00500708F043C0443600E0500708F438C0FC
:10020C0088249924AA24BB2411E0443F510718F0F8
:10021C00445F514007C004EF11E0041B150BA8010B
:10022C000AE0B02E483E03E0500720F0485E5340F1
:10023C00B394F8CF443600E0500720F044565040B9
:10024C00A394F8CF4A3018F04A509394FBCF042F64
:10025C00FBD0802E092DF8D0902E0A2DF5D0A02E93
:10026C000B2D003011F0F0D001C00FEFB02E08951F
:10027C0007EF802E902EA02EB02E08950EEF802E1C
:10028C00902EA02EB02E089510916700009166005C
:10029C004017510720F4509367004093660010916B
:1002AC006500009164000417150720F45093650055
:1002BC004093640020FC04C050916700409166009C
:1002CC0021FC04C05091650040916400413B04E066
:1002DC00500708F043C0443600E0500708F438C01B
:1002EC00CC24DD24EE24FF2411E0443F510718F008
:1002FC00445F514007C004EF11E0041B150BA8012B
:10030C000AE0F02E483E03E0500720F0485E5340D0
:10031C00F394F8CF443600E0500720F04456504098
:10032C00E394F8CF4A3018F04A50D394FBCF042F03
:10033C008BD0C02E0D2D88D0D02E0E2D85D0E02E3A
:10034C000F2D003011F080D001C00FEFF02E08956A
:10035C0007EFC02ED02EE02EF02E08950EEFC02EFB
:10036C00D02EE02EF02E089509ED02BF2A9509F447
:10037C0028E032BAAD98E6ECF1E0E20FF31D0994F7
:10038C0008C007C009C00DC010C012C014C018C0EE
:10039C001AC088BA909A1895092D0F7708BB919AB4
:1003AC001895A8BA939A1AD01895B8BA949A189521
:1003BC00C8BA959A18950D2D0F7708BB969A189573
:1003CC00E8BA979A1895F8BAAD9A01D01895119782
:1003DC0009F4AB98219709F4AC980895112703B34D
:1003EC00037002111FEF202E003091F01F3F79F4A3
:1003FC00033059F44091680050916900EBDE409154
:10040C006A0050916B0056DF0895E4DE53DF0895C7
:10041C000027009360000093610000936400009338
:10042C0065000FEF00936200009363000093660079
:10043C00009367000FEB802E902EA02EB02EC02EB6
:10044C00D02EE02EF02E08950B3008F00BE0F4E0E7
:10045C00E6E6E00FF31D04910895C0F9A4B099925B
:06046C0082F88090BF86BB
:00000001FF
